:100000000C9463000C948B000C948B000C948B006C
:100010000C948B000C948B000C948B000C948B0034
:100020000C948B000C948B000C948B000C94DA0EC7
:100030000C948B000C948B000C948B000C948B0014
:100040000C94380E0C948B000C94A80E0C94820E19
:100050000C948B000C948B000C948B000C948B00F4
:100060000C948B000C948B000000000024002700EF
:100070002A0000000000250028002B0000000000DE
:1000800023002600290004040404040404040202DA
:100090000202020203030303030301020408102007
:1000A0004080010204081020010204081020000012
:1000B0000008000201000003040700000000000027
:1000C0000000960F4F1211241FBECFEFD8E0DEBF05
:1000D000CDBF11E0A0E0B1E0ECE3F8E202C0059092
:1000E0000D92A832B107D9F722E0A8E2B1E001C031
:1000F0001D92A13AB207E1F710E0C2E6D0E004C0D9
:100100002197FE010E94E612C136D107C9F70E946D
:10011000D0100C9411140C940000833081F028F45A
:10012000813099F08230A9F008958730A9F08830A5
:10013000C9F08430B1F4809180008F7D03C080913C
:1001400080008F7780938000089584B58F7784BD79
:10015000089584B58F7DFBCF8091B0008F77809319
:10016000B00008958091B0008F7DF9CFCF93DF93D9
:10017000282F30E0F901E255FF4F8491F901E6564E
:10018000FF4FD491F901EA57FF4FC491CC23A1F05E
:1001900081110E948D00EC2FF0E0EE0FFF1FE4585C
:1001A000FF4FA591B491EC91ED2381E090E009F42B
:1001B00080E0DF91CF91089580E090E0FACF1F9327
:1001C000CF93DF93282F30E0F901E255FF4F849160
:1001D000F901E656FF4FD491F901EA57FF4FC49158
:1001E000CC23A9F0162F81110E948D00EC2FF0E096
:1001F000EE0FFF1FEE58FF4FA591B4918FB7F89403
:10020000EC91111108C0D095DE23DC938FBFDF91F4
:10021000CF911F910895DE2BF8CFCF93DF9390E01D
:10022000FC01E656FF4F24918A579F4FFC018491B1
:100230008823D1F090E0880F991FFC01E859FF4F07
:10024000A591B491FC01EE58FF4FC591D491611175
:100250000EC09FB7F8948C91E22FE0958E238C937B
:100260002881E223E8839FBFDF91CF9108958FB764
:10027000F894EC91E22BEC938FBFF6CF8E3008F020
:100280008E508770806480937C0080917A008064B7
:1002900080937A0080917A0086FDFCCF809178006F
:1002A0009091790008953FB7F894809163019091FF
:1002B0006401A0916501B091660126B5A89B05C0B7
:1002C0002F3F19F00196A11DB11D3FBFBA2FA92FD5
:1002D000982F8827BC01CD01620F711D811D911DD2
:1002E00042E0660F771F881F991F4A95D1F708953E
:1002F0008F929F92AF92BF92CF92DF92EF92FF9236
:100300000E9453014B015C0184E6C82ED12CE12CE4
:10031000F12C0E945301681979098A099B09683EEA
:10032000734081059105A8F321E0C21AD108E108C4
:10033000F10888EE880E83E0981EA11CB11CC11440
:10034000D104E104F10429F7FF90EF90DF90CF9002
:10035000BF90AF909F908F9008950895AF92BF92F5
:10036000CF92DF92EF92FF920F931F93CF93DF9381
:100370006C017B018B01040F151FEB015E01AE18B0
:10038000BF08C017D10759F06991D601ED91FC91D2
:100390000190F081E02DC6010995892B79F7C501FF
:1003A000DF91CF911F910F91FF90EF90DF90CF9051
:1003B000BF90AF900895FC01538D448D252F30E000
:1003C000842F90E0821B930B541710F0CF96089562
:1003D00001970895FC01918D828D981761F0A28D8F
:1003E000AE0FBF2FB11D5D968C91928D9F5F9F7355
:1003F000928F90E008958FEF9FEF0895FC01918D0B
:10040000828D981731F0828DE80FF11D858D90E077
:1004100008958FEF9FEF0895FC01918D228D892F14
:1004200090E0805C9F4F821B91098F7399270895FC
:1004300087E691E00E940C0221E0892B09F420E07C
:10044000822F089580E090E0892B29F00E94180205
:1004500081110C9400000895FC01A48DA80FB92F00
:10046000B11DA35ABF4F2C91848D90E001968F73DC
:100470009927848FA689B7892C93A089B1898C91FB
:10048000837080648C93938D848D981306C002884A
:10049000F389E02D80818F7D80830895EF92FF9214
:1004A0000F931F93CF93DF93EC0181E0888F9B8D97
:1004B0008C8D98131AC0E889F989808185FF15C051
:1004C0009FB7F894EE89FF896083E889F989808174
:1004D0008370806480839FBF81E090E0DF91CF9143
:1004E0001F910F91FF90EF900895F62E0B8D10E065
:1004F0000F5F1F4F0F731127E02E8C8D8E110CC0D4
:100500000FB607FCFACFE889F989808185FFF5CF1E
:10051000CE010E942C02F1CFEB8DEC0FFD2FF11DCF
:10052000E35AFF4FF0829FB7F8940B8FEA89FB895B
:1005300080818062CFCFCF93DF93EC01888D8823B9
:10054000B9F0AA89BB89E889F9898C9185FD03C036
:10055000808186FD0DC00FB607FCF7CF8C9185FF1B
:10056000F2CF808185FFEDCFCE010E942C02E9CF32
:10057000DF91CF910895CF93DF9300D0CDB7DEB751
:10058000DA012C91FB01308139832A83DC018D91C2
:100590009C91DC01ED91FC910284F385E02D22E039
:1005A00030E0AE014F5F5F4F61EF70E009950F9053
:1005B0000F90DF91CF9108956115710531F0FC0125
:1005C00080819181FB01918380830895CF92DF9296
:1005D000EF92FF920F931F93CF93DF93EC01162FAF
:1005E0006A017901E881F9810280F381E02D41E01F
:1005F00060EC0995E881F9810280F381E02D40E00B
:10060000612FCE010995E881F9810280F381E02D07
:10061000DE01A95FBE4F6C9181E0860F8C9340E0B4
:10062000CE0109958601EC0CFD1CE881F981028060
:10063000F381E02DE016F10639F0D8016D918D01BE
:1006400040E0CE010995F1CF41E060ECCE01099583
:100650008A819B81DC01ED91FC910680F781E02D80
:10066000DF91CF911F910F91FF90EF90DF90CF908E
:100670000994BF92CF92DF92EF92FF920F931F9354
:10068000CF93DF93EC01B62EC42ED22EE881F981F0
:100690000280F381E02D41E060EC0995E881F98169
:1006A0000280F381E02D40E06B2DCE010995E881B9
:1006B000F9810280F381E02D40E06C2DCE01099597
:1006C000E881F9810280F381E02D40E06D2DCE01BB
:1006D00009956801E00EF11EE881F9810280F3813D
:1006E000E02DEC14FD0439F0D6016D916D0140E070
:1006F000CE010995F1CF41E060ECCE0109958A81E8
:100700009B81DC01ED91FC910680F781E02DDF916A
:10071000CF911F910F91FF90EF90DF90CF90BF90FE
:100720000994DC0112968D919C91DC01ED91FC9174
:100730000190F081E02D0994CF93DF93DC01ED91DE
:10074000FC910480F581E02D442319F0DF91CF91D5
:100750000994EC01603C21F06B3D59F0CE01F6CFDD
:100760006BED0995E881F9810480F581E02D6CED50
:10077000F5CF6BED0995E881F9810480F581E02DD5
:100780006DEDECCF0F931F93CF93DF93EC01CA5F16
:10079000DE4F2881222321F06C3D49F06D3D09F1A7
:1007A000603C59F16B3D81F481E088833AC0DC0103
:1007B000AB5FBE4FEC9121E02E0F2C93E80FF92F89
:1007C000F11D20EC26831882FC01EB5FFE4F208197
:1007D00031E0320F3083820F911DDC0116966C934D
:1007E00020C0DC01AB5FBE4FEC9121E02E0F2C93BB
:1007F000E80FF92FF11D2BEDE5CF8C010B5F1E4F9C
:10080000D8014C91442351F0BC016A5F7F4FDC0159
:10081000ED91FC910680F781E02D0995F801108299
:100820001882DF91CF911F910F910895DC01ED9116
:10083000FC91309729F00280F381E02D0296099413
:100840000895FC01828D938D30E020E02817390750
:10085000E1F0A785B089A20FB31F4C91641312C0B9
:1008600080A591A52817390718F082A593A50895AA
:10087000220F331F858D968D280F391FF901808136
:10088000918108952F5F3F4FE1CF8585968508952B
:10089000CF93DF93EC01CD3C8CE0D807A0F42AE0A5
:1008A0002C9FC0012D9F900D112402960E94EC12E6
:1008B000FC01C193D193CF012197D7FD07C01182CD
:1008C00010823A96F9CF8FEF9FEFF0CFDF91CF9163
:1008D0000895EF92FF920F931F93CF93DF93EC0154
:1008E0008B0180E190E09F838E8381E088871D8665
:1008F000FB01E184F284C7010E94EC129983888392
:10090000892B61F1F801828193819B838A838481A1
:1009100095819D838C83868197819F838E8380853B
:100920008887FA86E986838594859C878B87858569
:100930008D8790E080E02B853C858217930770F4CB
:10094000E0913E02F0913F02E80FF91F2081E8811B
:10095000F981E80FF91F20830196EDCFDF91CF9148
:100960001F910F91FF90EF900895EF92FF920F93D8
:100970001F93CF93DF930097C1F1EC01FC013297F5
:10098000808191812AE0289F8001299F100D1124E8
:100990000C0F1D1F7801CE15DF0539F08AE0E81A2B
:1009A000F108C7010E941604F6CFC8018C1B9D0BED
:1009B000969587954DEC5CE4849F9001859F300D62
:1009C000949F300D11243F7746EF4203C001439FAF
:1009D000900D11240297800F911FDF91CF911F91ED
:1009E0000F91FF90EF900C948813DF91CF911F919E
:1009F0000F91FF90EF9008952F923F924F925F9248
:100A00006F927F928F929F92AF92BF92CF92DF921E
:100A1000EF92FF920F931F93CF93DF938C016B01A3
:100A2000FC01C481D58181859285C617D707B8F4AA
:100A3000C817D907A9F480E0DF91CF911F910F91DA
:100A4000FF90EF90DF90CF90BF90AF909F908F90EE
:100A50007F906F905F904F903F902F900895EB01A3
:100A6000F8012085211105C08C179D0738F081E021
:100A7000E3CF6E018C179D0708F46C011E012097CF
:100A800019F480E1282E312CC1010E9448043C0158
:100A9000009789F27C01512C412CF80180809180D3
:100AA000C414D504E9F05701A618B708C7010E947D
:100AB0001604E114F10469F0F401EA0DFB1D8191C3
:100AC0009191D7018D939D9388E001900D928A9525
:100AD000E1F7FFEF4F1A5F0A8AE0E80EF11CDDCF65
:100AE000C4010E94B504F8017182608221863286B9
:100AF00083859485C817D90708F0B9CFD487C387F1
:100B0000B6CF0F931F93CF93DF938C0160918F0229
:100B100070919002809191029091920286179707AE
:100B2000F8F420919102309192024AE0429FC00174
:100B3000439F900D1124C0918602D0918702C80F67
:100B4000D91FCE010E9416042097E9F480919102EA
:100B500090919202019690939202809391020EC01E
:100B600080918C0290918D02009741F0680F791F5F
:100B700086E892E00E94FC048111D3CFDF91CF91EF
:100B80001F910F910895F80181919191DE018D934C
:100B90009D9388E001900D928A95E1F7D7CF0F934E
:100BA0001F93CF93DF93EC018B0169857A8506173C
:100BB000170738F08E819F81680F791FCE010E9440
:100BC000FC0489859A852B853C850217130740F024
:100BD0008017910740F098012F5F3F4F3C872B878C
:100BE0000817190738F0CE010D96DF91CF911F91AC
:100BF0000F9108958AE0809F9001819F300D11240C
:100C000088819981820F931FF0CFAF92BF92CF92CC
:100C1000DF92EF92FF920F931F93CF93DF938C019C
:100C20007B01FC01C481D58181859285C617D707D8
:100C300078F4C817D90769F480E0DF91CF911F914C
:100C40000F91FF90EF90DF90CF90BF90AF900895FD
:100C5000EB01F8012085211105C08C179D0738F0A4
:100C600081E0EBCF7E018C179D0708F47C01209773
:100C700021F16E018FEF9FEFC115F0E4DF0718F44B
:100C8000C601880F991F0E94EC125C010097A1F227
:100C9000DC01F8018081918130E020E0E216F3066A
:100CA00081F0F901EE0FFF1FE80FF91F408151811C
:100CB0004D935D932F5F3F4FF1CF60E1C62ED12C56
:100CC000DFCF009711F00E948813F801B182A08253
:100CD000D286C18683859485C817D90708F6D4873C
:100CE000C387BECF0F931F93CF93DF93EC018B018C
:100CF00069857A850617170738F08E819F81680FFE
:100D0000791FCE010E94050689859A852B853C8531
:100D10000217130740F08017910740F098012F5FEA
:100D20003F4F3C872B870817190738F0CE010D96E7
:100D3000DF91CF911F910F910895000F111F8881AE
:100D40009981800F911FF4CF8F929F92AF92BF92A3
:100D5000CF92DF92EF92FF920F931F93CF93DF9387
:100D6000EC017B0189859A856817790760F0CE8050
:100D7000DF80C80ED91E0C811D810C151D0528F5BC
:100D80008017910719F589859A852B853C85E21690
:100D9000F30640F08E159F0548F097012F5F3F4FF7
:100DA0003C872B87E816F90608F458C0CE010D964B
:100DB000DF91CF911F910F91FF90EF90DF90CF9037
:100DC000BF90AF909F908F90089586012885211144
:100DD00027C080179107B8F60115110539F15801A0
:100DE000011580E4180730F5C501880F991F0E948E
:100DF000EC124C01009739F2DC018881998130E0D6
:100E000020E0C216D306C9F0F901EE0FFF1FE80F6C
:100E1000F91F408151814D935D932F5F3F4FF1CF7B
:100E20006C0108171907C0F66801D6CF60E1A62E3D
:100E3000B12CDACF8FEF9FEFDACF009711F00E943D
:100E4000881399828882BA86A9868B859C85081723
:100E5000190708F098CF1C870B8795CFEE0CFF1C65
:100E6000888199818E0D9F1DA3CFAF92BF92CF92A3
:100E7000DF92EF92FF920F931F93CF93DF938C013A
:100E80007B01DC011496CD91DC91159719968D911B
:100E90009C91C617D70778F4C817D90769F480E082
:100EA000DF91CF911F910F91FF90EF90DF90CF9046
:100EB000BF90AF900895EB01F8012085211105C086
:100EC0008C179D0738F081E0EBCF7E018C179D07D2
:100ED00008F47C016E01209719F480E1C82ED12C12
:100EE000C6010E94EC125C010097C9F2FC01D80116
:100EF0008D919C9130E020E0E216F30641F0DC0198
:100F0000A20FB31F4C9141932F5F3F4FF5CF009736
:100F100011F00E948813F801B182A082C186D286A6
:100F200083859485C817D90770F6D487C387CBCF3C
:100F3000CF93FC0183859485C0E06817790750F54D
:100F40008385948501976817790778F4808191816A
:100F50009B012F5F3F4FDC01A20FB31F4C91680F25
:100F6000791FDB014C93B901EBCF94878387C08550
:100F7000CC2399F04185528526813781BA01621BC5
:100F8000730B8617970730F42417350718F4CF0131
:100F90000E9435078C2FCF910895C1E0FBCF0F93AE
:100FA0001F93CF93DF93EC018B0169857A858B8545
:100FB0009C8586179707A8F4F8018081E881F9815C
:100FC0002B853C85E20FF31F80832B853C85C9016F
:100FD00001969C878B87C901DF91CF911F910F915B
:100FE00008958E819F81009719F48FEF9FEFF4CFC2
:100FF000680F791FCE010E9435078111DDCFF5CF33
:101000000F931F93CF93DF93EC018B0169857A8552
:101010000617170738F08E819F81680F791FCE0160
:101020000E94350789859A852B853C850217130711
:1010300040F08017910740F098012F5F3F4F3C87A9
:101040002B870817190738F0CE010D96DF91CF9145
:101050001F910F91089588819981800F911FF6CF7C
:10106000CF92DF92FF920F931F93CF93DF938C0168
:10107000F62ED0E0C0E06C018FE0C80ED11CF80164
:10108000828D938DC817D90798F4BE01C6010E94BE
:101090000008FC0180818F1109C0CE01DF91CF9142
:1010A0001F910F91FF90DF90CF9008952196E7CF89
:1010B0008FEF9FEFF3CFCF92DF92EF92FF920F93DC
:1010C0001F93CF93DF931F92CDB7DEB78C01698357
:1010D000F12CE12C6C018FE0C80ED11CF801828D3F
:1010E000938DE816F90698F4B701C6010E9400082E
:1010F000FC0190818981981306C0B701C8014D9603
:101100000E94A4060EC0FFEFEF1AFF0AE7CFBE0150
:101110006F5F7F4FC6010E94CF0797FF0CC0C801C9
:101120000D960F90DF91CF911F910F91FF90EF904F
:10113000DF90CF900895F801208131812F5F3F4FDC
:1011400031832083BC01DACFCF92DF92EF92FF92FE
:101150000F931F93CF93DF938C01D62ED0E0C0E086
:101160007C018FE0E80EF11CD8015A968D919C917C
:10117000C817D90708F052C0BE01C7010E94000875
:10118000FC0180818D1148C0D80198968D919C9169
:10119000C817D90798F5AE01440F551FBE01019736
:1011A000FA0132966817790790F4D8015D962D916F
:1011B0003C916F5F7F4FD901AE0FBF1FCD90DC9088
:1011C000240F351FD901CD92DC92AF01E9CFF80190
:1011D00091A780A725A1222389F046A157A123A189
:1011E00034A1BA01621B730B8617970738F42417D2
:1011F000350720F4C8014D960E940506BE01C701BF
:101200000E949807CE01DF91CF911F910F91FF901F
:10121000EF90DF90CF9008952196A6CF8FEF9FEFAC
:10122000F2CFCF92DF92EF92FF920F931F93CF9363
:10123000DF931F92CDB7DEB78C016983F12CE12CCF
:101240006C018FE0C80ED11CF801828D938DE816D9
:10125000F90698F4B701C6010E940008FC019081CC
:101260008981981306C0B701C8014D960E94720685
:101270000EC0FFEFEF1AFF0AE7CFBE016F5F7F4F8F
:10128000C6010E94CF0797FF0CC0C8010D960F90B2
:10129000DF91CF911F910F91FF90EF90DF90CF9052
:1012A0000895F801208131812F5F3F4F31832083E2
:1012B000BC01DACFCF92DF92EF92FF920F931F9390
:1012C000CF93DF931F92CDB7DEB78C016983F12CEA
:1012D000E12C6C018EE0C80ED11CF801818D928D3D
:1012E000E816F90698F4B701C6010E940008FC014F
:1012F00090818981981306C0B701C8014C960E945D
:1013000000080EC0FFEFEF1AFF0AE7CFBE016F5FC4
:101310007F4FC6010E94CF0797FF0CC0C8010D96F2
:101320000F90DF91CF911F910F91FF90EF90DF9081
:10133000CF900895F801208131812F5F3F4F318395
:101340002083BC01DACFFC0180819181009711F0EC
:101350000C94881308952F923F925F926F927F9220
:101360008F929F92AF92BF92CF92DF92EF92FF92B5
:101370000F931F93CF93DF93CDB7DEB729970FB6A7
:10138000F894DEBF0FBECDBF6C017B01DB016C9119
:1013900011965C90673008F05CC4E62FF0E0ED52E7
:1013A000F64F0C94E612DA09110ADE0B4C0C8B0C8A
:1013B0002A0D660DDC01ED91FC910084F185E02D94
:1013C000423011F1F12CE12C10E000E023E030E09C
:1013D000452D60E0C601099529960FB6F894DEBF49
:1013E0000FBECDBFDF91CF911F910F91FF90EF9076
:1013F000DF90CF90BF90AF909F908F907F906F9035
:101400005F903F902F90089519821A8283E08B831A
:1014100033E0E32EF12C8E010F5F1F4F30E020E010
:10142000D7CFEDB7FEB7F987E887443079F0DC0114
:10143000ED91FC910084F185E02DF12CE12C10E080
:1014400000E023E030E0452D61E0C4CFF7011281D8
:101450008381282E312CD6011496ED90FC90823099
:1014600009F4E3C030F5882309F423C1813009F47D
:10147000CCC0612FC7010E945B08DC012D923C9219
:101480001982D601ED91FC910084F185E02DEE24C6
:10149000E394F12C8E010F5F1F4F30E020E0452DCB
:1014A00061E0C60109950FB6F894DEBF0FBECDBF4F
:1014B00093CF843009F4C6C008F4BCC08530C9F6A7
:1014C0005701F6E5AF0EB11C712C612CC701805994
:1014D0009F4F9F838E8345019FE0890E911CAE81B3
:1014E000BF818D919C916816790650F4B301C401B7
:1014F0000E940008FC0180811813B1C077FEB3C0C0
:1015000083E090E00E94EC124C0180914C018C3001
:1015100008F0CBC091E0980F90934C01D4018C93CC
:1015200090E0FC01EE0FFF1FE80FF91FE85DFE4F92
:1015300088EB9BE092838183612FC5010E94110992
:10154000DC018D929C92612FC5010E941109FC0162
:10155000A080B180D5018C918C3008F08ACF61E0F9
:10156000812F0E940D01F5018081282F30E0F901C3
:10157000EE0FFF1FE20FF31FE85DFE4F9081907C9E
:10158000212F2F73922B9083D50111961C921197C6
:1015900012961C922CE0622F0E94DA12829FB001F8
:1015A000112430E020E0AB01420F531FFA01EE0F8F
:1015B000FF1FE40FF51FE85DFE4F908196FD16C0FA
:1015C0002F5F3F4F2C30310571F781110FC0109202
:1015D000800082E080938100109285001092840048
:1015E000B19A80916F00826080936F00D501EC9179
:1015F0008E2F90E0FC01EE0FFF1FE80FF91FE85D52
:10160000FE4F80818064808334CF60E0812F0E9410
:101610000D01812F0E94B600082F612FC7018C9603
:101620000E945A09FC01008324CF61E0812F0E94AF
:101630000D011FCF60E0812F0E940D01812F0E94BC
:101640003E0117CF61E0812F0E940D0161E0812FE3
:101650000E940D0160E0812F0E94DF000ACFFFEFA2
:101660006F1A7F0A3CCF612FC5010E941109DC016E
:10167000ED91FC91E0818E2F90E0FC01EE0FFF1FB9
:10168000E80FF91FE85DFE4F80818F7B8083612F1B
:10169000C5010E941109FC01808191810E9488137B
:1016A000612FC5010E94A4082BCF8FEFF401808326
:1016B00043CFB12CA12CF701E059FF4FFF83EE83FC
:1016C0004701F6E58F0E911C34012FE0620E711C6C
:1016D000AE81BF818D919C91A816B90650F4B501D9
:1016E000C3010E940008FC01808118131EC0B7FED0
:1016F00020C0B12CA12C3701F5E46F0E711C4701FD
:101700002AE3820E911CD3018D919C91A816B906F3
:1017100050F4B501C4010E940008FC018081181337
:101720002AC0B7FE2CC060E081CFFFEFAF1ABF0A1E
:10173000CFCF612FC4010E941109DC01ED91FC9112
:10174000E0818E2F90E0FC01EE0FFF1FE80FF91FE4
:10175000E85DFE4F80818F7B8083612FC4010E94F2
:101760001109FC01808191810E948813612FC401BD
:101770000E94A408BECFFFEFAF1ABF0AC4CFB12C9E
:10178000A12CD3018D919C91A816B90660F6B501E4
:10179000C4010E940008FC01808118130BC0B50130
:1017A000C701885B9F4F0E949807B501C4010E9442
:1017B0009807B9CFFFEFAF1ABF0AE3CF443079F0F3
:1017C000DC01ED91FC910084F185E02DF12CE12C00
:1017D00010E000E023E030E0452D62E0FBCDF701B2
:1017E00012819380DC011496ED90FC90612FC7016B
:1017F0000E9430080196C9F1612FC7010E945B0861
:10180000FC0180819181029709F042C001E09110B2
:1018100001C000E0602F812F0E94DF00912C812CFD
:101820003701FDE86F0E711C22E8E20EF11CD301B6
:101830008D919C918816990668F5B401C7010E94A4
:10184000CF051C830983DC01ED91FC910480F581B7
:10185000E02DAE014F5F5F4FBE016C5F7F4F029680
:101860000995BFEF8B1A9B0AE2CF81E08D83D601E9
:10187000ED91FC910084F185E02DEE24E394F12CB0
:101880008E010B5F1F4F30E020E0452D62E009CE56
:1018900083E0ECCF80E0EACF433079F0DC01ED91DA
:1018A000FC910084F185E02DF12CE12C10E000E0AA
:1018B00023E030E0452D63E08DCDF7011281612FEB
:1018C000DC0114968D919C910E9421040097F1F007
:1018D00001970297F0F4812F0E94B60021E0892B36
:1018E00009F420E080E089832A83D601ED91FC9100
:1018F0000084F185E02D02E0E02EF12C8E010F5FD7
:101900001F4F30E020E0452D63E0CBCD81E020E0AB
:10191000EACF82E0FCCF443079F0DC01ED91FC911C
:101920000084F185E02DF12CE12C10E000E023E0B3
:1019300030E0452D64E04ECDF7011281DC011496B4
:101940008D909C90612FC4010E942104009799F40E
:1019500081E08983D601ED91FC910084F185E02D31
:10196000EE24E394F12C8E010F5F1F4F30E020E056
:10197000452D64E096CD049711F083E0EACFF7019E
:101980000381612FC4010E943008019609F3612F81
:10199000C4010E945B08DC018D919C91049769F75A
:1019A000E02EF12C61E0812F0E940D01E114F10481
:1019B00029F460E0812F0E94DF002BC0BFEFEB16FF
:1019C000F10411F461E0F6CFE12FF0E0E255FF4FB2
:1019D000E491E33029F148F4E130B9F0E230D9F094
:1019E000E0E8EE16F10474F7E4CFE73019F1E830DF
:1019F00049F1E430A9F780918000806280938000F3
:101A0000F0928B00E0928A0004C084B5806884BDA7
:101A100007BD80E09ECF84B5806284BD08BDF9CF4C
:101A200080918000806880938000F0928900E0922D
:101A30008800EFCF8091B00080688093B000009361
:101A4000B300E7CF8091B00080628093B000009334
:101A5000B400DFCF433079F0DC01ED91FC910084DC
:101A6000F185E02DF12CE12C10E000E023E030E0E6
:101A7000452D65E0AFCCF7011281612FDC01149692
:101A80008D919C910E9421040097E1F0039722E040
:101A90000297C8F4812F0E943E0120E029839A8397
:101AA0008B83D601ED91FC910084F185E02DB3E0AC
:101AB000EB2EF12C8E010F5F1F4F30E020E0452D03
:101AC00065E0EFCC21E080E090E0E8CF443079F0B1
:101AD000DC01ED91FC910084F185E02DF12CE12CED
:101AE00010E000E023E030E0452D66E073CCF70124
:101AF0001281DC0114968D909C90612FC4010E948C
:101B00002104009799F481E08983D601ED91FC913D
:101B10000084F185E02DEE24E394F12C8E010F5F1B
:101B20001F4F30E020E0452D66E0BBCC059709F063
:101B30008CC0F701038184E0053B30F7612FC401BD
:101B40000E94300897FDDFCF612FC4010E945B081F
:101B5000DC018D919C91059709F079C0B6E58B0E5B
:101B6000911C612FC4010E941109DC01ED91FC91CF
:101B7000E0818E2F90E0FC01EE0FFF1FE80FF91FB0
:101B8000E85DFE4F808186FFBECF612FC4010E94B9
:101B90001109DC01ED91FC9110811C3008F053C05B
:101BA000828148E5842E42E0942E881A910887FDB0
:101BB00093941401220C331C220C331C818168E89D
:101BC000E62EF12CE81AF10887FDF394EE0CFF1CC9
:101BD000EE0CFF1C37010F2C000C880899089101AE
:101BE000032C000C440B550B2619370948095909D9
:101BF000A02FB0E00E949E1224EB30E040E050E0C5
:101C00000E947F12BA01A901460D571D681D791D5A
:101C10004E155F052CF07101421553050CF47A0145
:101C2000B2E0EB1AF108EE0CFF1C2FB7F894812FED
:101C300090E0FC01EE0FFF1FE80FF91FE85DFE4F7B
:101C4000F282E1822FBF80E05FCF82E05DCF83E050
:101C50005BCFDC01ED91FC910084F185E02DF12C4E
:101C6000E12C10E000E022E030E0452D0995B4CBF6
:101C70001F920F920FB60F9211242F933F938F93C1
:101C80009F93AF93BF9380915F0190916001A0916A
:101C90006101B091620130915E0123E0230F2D3785
:101CA00058F50196A11DB11D20935E0180935F013F
:101CB00090936001A0936101B093620180916301F0
:101CC00090916401A0916501B09166010196A11DFA
:101CD000B11D8093630190936401A0936501B0935B
:101CE0006601BF91AF919F918F913F912F910F907E
:101CF0000FBE0F901F90189526E8230F0296A11D86
:101D0000B11DD2CF1F920F920FB60F9211242F93B5
:101D10003F934F935F936F937F938F939F93AF9373
:101D2000BF93EF93FF9387E691E00E942C02FF910F
:101D3000EF91BF91AF919F918F917F916F915F9143
:101D40004F913F912F910F900FBE0F901F901895BC
:101D50001F920F920FB60F9211242F938F939F9380
:101D6000EF93FF93E0917701F09178018081E0910A
:101D70007D01F0917E0182FD1BC0908180918001E8
:101D80008F5F8F7320918101821741F0E091800174
:101D9000F0E0E959FE4F958F80938001FF91EF911C
:101DA0009F918F912F910F900FBE0F901F901895BC
:101DB0008081F4CF1F920F920FB60F9211242F93B0
:101DC0003F934F935F936F937F938F939F93AF93C3
:101DD000BF93CF93DF93EF93FF9380914D01C09119
:101DE0004C01D0E087FF24C010928500109284003F
:101DF00080914D018F5F80934D0180914D01082EA0
:101E0000000C990B8C179D0724F480914D018C30A8
:101E1000C4F18091840090918500049680349C499F
:101E200008F47AC08091840090918500049676C071
:101E300080914D01082E000C990B8C179D07C4F65C
:101E4000E0914D018E2FEE0F990BFC01EE0FFF1F5D
:101E5000E80FF91FE85DFE4F808186FFC9CFE09152
:101E60004D018E2FEE0F990BFC01EE0FFF1FE80FB7
:101E7000F91FE85DFE4F808160E08F730E94DF00F4
:101E8000B7CF2091840030918500E0914D018E2FD5
:101E9000EE0F990BFC01EE0FFF1FE80FF91FE85D35
:101EA000FE4F81819281820F931F909389008093CE
:101EB0008800E0914D018E2FEE0F990BFC01EE0F83
:101EC000FF1FE80FF91FE85DFE4F808186FF11C0FC
:101ED000E0914D018E2FEE0F990BFC01EE0FFF1FCD
:101EE000E80FF91FE85DFE4F808161E08F730E946B
:101EF000DF00FF91EF91DF91CF91BF91AF919F9163
:101F00008F917F916F915F914F913F912F910F90A2
:101F10000FBE0F901F90189580E49CE99093890064
:101F2000809388008FEF80934D01E3CFCF92DF92B3
:101F3000FF920F931F93CF93DF93E7E6F1E01382B5
:101F4000128288EE93E0A0E0B0E084839583A683BC
:101F5000B7838AE191E09183808385EC90E0958757
:101F6000848784EC90E09787868780EC90E0918B63
:101F7000808B81EC90E0938B828B82EC90E0958B50
:101F8000848B86EC90E0978B868B118E128E138E4D
:101F9000148EC4E0D2E000E110E01F830E83CC2455
:101FA000CA94DC2CD986C8861B870A87FF24F39441
:101FB000FC861E861D861A8B098BDC8ACB8A1E8BBB
:101FC0000D8BFF8A1C8E1B8E1A8E198F088F80E155
:101FD00090E00E94EC12988B8F8718A30F8FDAA2E3
:101FE000C9A21CA30BA3FDA21BA61AA619A618A67C
:101FF0001FA30EA380E290E00E94EC129E8F8D8FB3
:10200000198218821D830C831BAB0AABDDAACCAAF4
:102010001FAB0EABF8AE19AE1DAF0CAFDFAECEAE40
:102020001093450200934402F092460210924B0234
:1020300010924A02109249021093480200934702FC
:1020400080E190E00E94EC129BAF8AAF10934F02A8
:1020500000934E02D0925102C0925002109353024C
:1020600000935202F09254021092590210925802B8
:1020700010925702109356020093550280E190E0AF
:102080000E94EC1290934D0280934C021DA61CA658
:1020900019AB08AB1093610200936002D092630207
:1020A000C09262021093650200936402F09266028D
:1020B000109268021092670210936C0200936B02F8
:1020C000D0926E02C0926D021093700200936F0264
:1020D000F0927102109276021092750210927402C0
:1020E000109373020093720280E190E00E94EC1260
:1020F00090936A028093690210937A0200937902A6
:10210000D0927C02C0927B0210937E0200937D02EB
:10211000F0927F0210928502109284021092830244
:1021200010928202109381020093800280E290E07C
:102130000E94EC12909378028093770210925B02D7
:1021400010925A0210935F0200935E02109389026C
:1021500000938802D0928B02C0928A0210938D0263
:1021600000938C02F0928E021092940210929302CD
:1021700010929202109291021093900200938F029B
:1021800080E190E00E944804909387028093860249
:10219000DF91CF911F910F91FF90DF90CF90089525
:1021A000CF93DF93CDB7DEB760970FB6F894DEBF5D
:1021B0000FBECDBF789484B5826084BD84B5816044
:1021C00084BD85B5826085BD85B5816085BD809102
:1021D0006E00816080936E0010928100809181007A
:1021E0008260809381008091810081608093810072
:1021F000809180008160809380008091B100846034
:102200008093B1008091B00081608093B000809194
:102210007A00846080937A0080917A008260809353
:102220007A0080917A00816080937A0080917A00B0
:10223000806880937A001092C10088E091E00E944B
:10224000EC128C018AE091E0D80111969C938E9358
:1022500087E691E013969C938E93129784E092E028
:1022600015969C938E931497F801EB5FFE4F1082A6
:10227000319610823196108280915401811115C0DF
:102280008CED92E090934F0180934E018DEA91E0A6
:1022900090935101809350018BEB92E09093530106
:1022A0008093520181E0809354018EE491E09A83FF
:1022B00089831C830B83CE0101960E948105CE0188
:1022C00001960E94160410935D0100935C0161E089
:1022D0008DE00E940D0161E08DE00E94DF000E9410
:1022E000780160E08DE00E94DF000E94780161E0EB
:1022F0008DE00E94DF000E94780160E08DE00E9486
:10230000DF0060E08DE00E940D01D8011296ED9192
:10231000FC91A089B18982E08C93A485B5851C923B
:10232000A685B78580E18C93108EA489B58986E057
:102330008C93A289B3898C9180618C93A289B38993
:102340008C9188608C93A289B3898C9180688C93DE
:102350000288F389E02D80818F7D80830E9478013F
:1023600030E020E050E040E060EF70E0C8010E9403
:10237000E60280E0A82E80E0B82E6EE372E0CE0187
:1023800001960E946904F12CE12C8C859D85E8164C
:10239000F90608F04FC0B701CE0101960E9400086F
:1023A000FC011081612F84E092E00E945B08DC0157
:1023B0008D919C910197D1F5812F0E94B600082F35
:1023C000612F80E392E00E945A09FC018081081786
:1023D00069F1612F80E392E00E945A09DC010C93BD
:1023E000D12CC12C8091910290919202C816D906ED
:1023F000E8F4B60186E892E00E94CF05188B21E050
:10240000013009F020E02F87DC01ED91FC91048080
:10241000F581E02DAE01415F5F4FBE01605F7F4FF0
:1024200002960995BFEFCB1ADB0ADCCFEFEFEE1A6D
:10243000FE0AABCFCE0101960E94A30900915C0178
:1024400010915D01D80112968D919C91DC01ED9166
:10245000FC910084F185E02D0995892BA1F0F8010C
:1024600082819381DC01ED91FC910284F385E02D62
:102470000995D801ED91FC910190F081E02D682F34
:10248000C8010995DFCFA114B10409F476CF0E94E9
:102490001802882309F471CF0E9400006ECF80914A
:1024A000860290918702009731F00E94B504109245
:1024B00087021092860283E992E00E9416048091BE
:1024C000770290917802009711F00E94881389E6B4
:1024D00092E00E94A3098CE492E00E94A3098EE39B
:1024E00092E00E94A309809121029091220200971C
:1024F00011F00E94881383E192E00C94A309052E49
:1025000097FB1EF400940E94961257FD07D00E947C
:10251000A91207FC03D04EF40C94961250954095E6
:10252000309521953F4F4F4F5F4F0895909580957F
:10253000709561957F4F8F4F9F4F08950E94CB12EA
:10254000A59F900DB49F900DA49F800D911D112407
:102550000895A1E21A2EAA1BBB1BFD010DC0AA1FE4
:10256000BB1FEE1FFF1FA217B307E407F50720F0FC
:10257000A21BB30BE40BF50B661F771F881F991F77
:102580001A9469F760957095809590959B01AC01C0
:10259000BD01CF010895A29FB001B39FC001A39FC9
:1025A000700D811D1124911DB29F700D811D11248C
:1025B000911D0895991B79E004C0991F961708F0A2
:1025C000961B881F7A95C9F780950895EE0FFF1F17
:1025D0000590F491E02D09940F931F93CF93DF930F
:1025E0008230910510F482E090E0E0919F02F0913A
:1025F000A00230E020E0B0E0A0E0309799F421158F
:10260000310509F44AC0281B390B24303105D8F5AF
:102610008A819B816115710589F1FB019383828316
:10262000FE0111C040815181028113814817590771
:10263000E0F04817590799F4109761F012960C933F
:10264000129713961C933296CF01DF91CF911F9171
:102650000F91089500939F021093A002F4CF2115CB
:10266000310551F04217530738F0A901DB019A01F7
:10267000BD01DF01F801C1CFEF01F9CF9093A002B6
:1026800080939F02CDCFFE01E20FF31F81939193C0
:102690002250310939832883D7CF20919D02309170
:1026A0009E02232B41F420910201309103013093CB
:1026B0009E0220939D02209100013091010121157D
:1026C000310541F42DB73EB7409104015091050109
:1026D000241B350BE0919D02F0919E02E217F30757
:1026E000A0F42E1B3F0B2817390778F0AC014E5F82
:1026F0005F4F2417350748F04E0F5F1F50939E021F
:1027000040939D02819391939FCFF0E0E0E09CCFB6
:10271000CF93DF930097E9F0FC0132971382128286
:10272000A0919F02B091A002ED0130E020E010974F
:10273000A1F420813181820F931F20919D0230915D
:102740009E022817390709F061C0F0939E02E093BA
:102750009D02DF91CF910895EA01CE17DF07E8F5DA
:102760004A815B819E0141155105B1F7E901FB8367
:10277000EA8349915991C40FD51FEC17FD0761F405
:10278000808191810296840F951FE9019983888346
:10279000828193819B838A83F0E0E0E012968D91A1
:1027A0009C9113970097B9F52D913C911197CD010C
:1027B0000296820F931F20919D0230919E0228174E
:1027C000390739F6309751F51092A00210929F0206
:1027D000B0939E02A0939D02BCCFD383C28340815D
:1027E0005181840F951FC817D90761F44E5F5F4F61
:1027F00088819981480F591F518340838A819B8129
:10280000938382832115310509F0B0CFF093A002A4
:10281000E0939F029ECFFD01DC01C0CF13821282A4
:10282000D7CF10E0C2E6D0E004C0FE010E94E6125D
:0C2830002196C336D107C9F7F894FFCFFA
:10283C000000A102800000000000C2039C03910371
:10284C00AB093903E602000000004E02AE01DB01C9
:08285C009B020C02EA01FE01DF
:00000001FF
